BL51 BANKED LINKER/LOCATER V6.05                                                        08/19/2015  12:09:32  PAGE 1


BL51 BANKED LINKER/LOCATER V6.05, INVOKED BY:
C:\KEIL\C51\BIN\BL51.EXE 1602-miaobiao.obj TO 1602-miaobiao


MEMORY MODEL: SMALL


INPUT MODULES INCLUDED:
  1602-miaobiao.obj (1602_MIAOBIAO)
  C:\KEIL\C51\LIB\C51S.LIB (?C_STARTUP)
  C:\KEIL\C51\LIB\C51S.LIB (?C_INIT)


LINK MAP OF MODULE:  1602-miaobiao (1602_MIAOBIAO)


            TYPE    BASE      LENGTH    RELOCATION   SEGMENT NAME
            -----------------------------------------------------

            * * * * * * *   D A T A   M E M O R Y   * * * * * * *
            REG     0000H     0008H     ABSOLUTE     "REG BANK 0"
            DATA    0008H     0010H     UNIT         ?DT?1602_MIAOBIAO
            IDATA   0018H     0001H     UNIT         ?STACK

            * * * * * * *   C O D E   M E M O R Y   * * * * * * *
            CODE    0000H     0003H     ABSOLUTE     
            CODE    0003H     0007H     UNIT         ?PR?_LCD_POS?1602_MIAOBIAO
                    000AH     0001H                  *** GAP ***
            CODE    000BH     0003H     ABSOLUTE     
            CODE    000EH     0107H     UNIT         ?PR?MAIN?1602_MIAOBIAO
            CODE    0115H     008CH     UNIT         ?C_C51STARTUP
            CODE    01A1H     0088H     UNIT         ?CO?1602_MIAOBIAO
            CODE    0229H     0066H     UNIT         ?PR?PLAY?1602_MIAOBIAO
            CODE    028FH     0055H     UNIT         ?PR?TIME0?1602_MIAOBIAO
            CODE    02E4H     002CH     UNIT         ?PR?LCD_INIT?1602_MIAOBIAO
            CODE    0310H     0023H     UNIT         ?PR?_DELAY1?1602_MIAOBIAO
            CODE    0333H     001FH     UNIT         ?PR?_LCD_WDAT?1602_MIAOBIAO
            CODE    0352H     001BH     UNIT         ?PR?_LCD_WCMD?1602_MIAOBIAO
            CODE    036DH     0017H     UNIT         ?C_INITSEG
            CODE    0384H     0012H     UNIT         ?PR?BEEP?1602_MIAOBIAO
            CODE    0396H     000AH     UNIT         ?PR?_DELAY?1602_MIAOBIAO



OVERLAY MAP OF MODULE:   1602-miaobiao (1602_MIAOBIAO)


SEGMENT
  +--> CALLED SEGMENT
---------------------
?C_C51STARTUP
  +--> ?PR?MAIN?1602_MIAOBIAO
  +--> ?C_INITSEG

?PR?MAIN?1602_MIAOBIAO
  +--> ?PR?LCD_INIT?1602_MIAOBIAO
  +--> ?PR?_LCD_POS?1602_MIAOBIAO
  +--> ?PR?_LCD_WDAT?1602_MIAOBIAO
BL51 BANKED LINKER/LOCATER V6.05                                                      08/19/2015  12:09:32  PAGE 2


  +--> ?CO?1602_MIAOBIAO
  +--> ?PR?_DELAY1?1602_MIAOBIAO
  +--> ?PR?BEEP?1602_MIAOBIAO
  +--> ?PR?PLAY?1602_MIAOBIAO

?PR?LCD_INIT?1602_MIAOBIAO
  +--> ?PR?_DELAY1?1602_MIAOBIAO
  +--> ?PR?_LCD_WCMD?1602_MIAOBIAO

?PR?_DELAY1?1602_MIAOBIAO
  +--> ?PR?_LCD_WCMD?1602_MIAOBIAO

?PR?_LCD_WCMD?1602_MIAOBIAO
  +--> ?PR?_DELAY?1602_MIAOBIAO

?PR?_LCD_POS?1602_MIAOBIAO
  +--> ?PR?_LCD_WCMD?1602_MIAOBIAO

?PR?_LCD_WDAT?1602_MIAOBIAO
  +--> ?CO?1602_MIAOBIAO
  +--> ?PR?_DELAY?1602_MIAOBIAO

?PR?BEEP?1602_MIAOBIAO
  +--> ?PR?_DELAY?1602_MIAOBIAO

?PR?PLAY?1602_MIAOBIAO
  +--> ?PR?_LCD_POS?1602_MIAOBIAO
  +--> ?PR?_LCD_WDAT?1602_MIAOBIAO



SYMBOL TABLE OF MODULE:  1602-miaobiao (1602_MIAOBIAO)

  VALUE           TYPE          NAME
  ----------------------------------

  -------         MODULE        1602_MIAOBIAO
  C:0000H         SYMBOL        _ICE_DUMMY_
  D:0080H         PUBLIC        P0
  D:00A0H         PUBLIC        P2
  D:00B0H         PUBLIC        P3
  B:00B0H.0       PUBLIC        S2
  B:00B0H.1       PUBLIC        S3
  B:00A8H.7       PUBLIC        EA
  B:00A0H.3       PUBLIC        BEEP
  C:0384H         PUBLIC        beep
  C:000EH         PUBLIC        main
  B:00A0H.6       PUBLIC        dula
  B:00A0H.7       PUBLIC        wela
  D:0008H         PUBLIC        display2
  D:0089H         PUBLIC        TMOD
  D:0010H         PUBLIC        KeyCount
  C:0229H         PUBLIC        play
  C:028FH         PUBLIC        Time0
  C:0352H         PUBLIC        _lcd_wcmd
  C:0319H         PUBLIC        _delay1
  C:0339H         PUBLIC        _lcd_wdat
BL51 BANKED LINKER/LOCATER V6.05                                                      08/19/2015  12:09:32  PAGE 3


  B:00B0H.4       PUBLIC        LCD_EN
  B:00A8H.1       PUBLIC        ET0
  C:02E4H         PUBLIC        lcd_init
  D:008CH         PUBLIC        TH0
  D:008AH         PUBLIC        TL0
  C:01A1H         PUBLIC        cdis1
  B:0088H.4       PUBLIC        TR0
  C:01B2H         PUBLIC        cdis2
  C:01C3H         PUBLIC        cdis3
  B:00B0H.5       PUBLIC        LCD_RS
  C:01D4H         PUBLIC        cdis4
  C:01E5H         PUBLIC        cdis5
  C:01F6H         PUBLIC        cdis6
  C:0207H         PUBLIC        cdis7
  B:00B0H.6       PUBLIC        LCD_RW
  C:0218H         PUBLIC        cdis8
  C:0003H         PUBLIC        _lcd_pos
  C:0396H         PUBLIC        _Delay
  D:0011H         PUBLIC        display
  -------         PROC          _DELAY
  D:0006H         SYMBOL        num
  C:0396H         LINE#         70
  C:0396H         LINE#         71
  C:0396H         LINE#         72
  C:039FH         LINE#         73
  -------         ENDPROC       _DELAY
  -------         PROC          BEEP
  -------         DO            
  D:0005H         SYMBOL        y
  -------         ENDDO         
  C:0384H         LINE#         78
  C:0384H         LINE#         79
  C:0384H         LINE#         81
  C:0386H         LINE#         82
  C:0386H         LINE#         83
  C:0388H         LINE#         84
  C:038FH         LINE#         85
  C:0393H         LINE#         86
  C:0395H         LINE#         87
  -------         ENDPROC       BEEP
  C:0310H         SYMBOL        L?0072
  C:0312H         SYMBOL        L?0073
  -------         PROC          L?0071
  -------         ENDPROC       L?0071
  C:0310H         SYMBOL        L?0072
  C:0312H         SYMBOL        L?0073
  -------         PROC          _DELAY1
  D:0006H         SYMBOL        ms
  -------         DO            
  D:0005H         SYMBOL        n
  -------         ENDDO         
  C:0319H         LINE#         92
  C:0319H         LINE#         93
  C:0319H         LINE#         95
  C:0323H         LINE#         96
  C:0323H         LINE#         97
  C:032BH         LINE#         98
BL51 BANKED LINKER/LOCATER V6.05                                                      08/19/2015  12:09:32  PAGE 4


  C:032BH         LINE#         99
  C:032CH         LINE#         100
  C:032DH         LINE#         101
  C:032EH         LINE#         102
  C:032FH         LINE#         103
  C:0332H         LINE#         104
  C:0332H         LINE#         105
  -------         ENDPROC       _DELAY1
  -------         PROC          _LCD_WCMD
  D:0007H         SYMBOL        cmd
  C:0352H         LINE#         113
  C:0352H         LINE#         114
  C:0352H         LINE#         116
  C:0354H         LINE#         118
  C:0356H         LINE#         119
  C:0357H         LINE#         120
  C:0358H         LINE#         121
  C:035AH         LINE#         122
  C:035EH         LINE#         123
  C:0360H         LINE#         124
  C:0364H         LINE#         125
  C:0366H         LINE#         126
  -------         ENDPROC       _LCD_WCMD
  -------         PROC          L?0074
  -------         ENDPROC       L?0074
  -------         PROC          _LCD_WDAT
  D:0007H         SYMBOL        dat
  C:0339H         LINE#         135
  C:0339H         LINE#         136
  C:0339H         LINE#         138
  C:033BH         LINE#         140
  C:033DH         LINE#         141
  C:033FH         LINE#         142
  C:0343H         LINE#         143
  C:0345H         LINE#         144
  C:0349H         LINE#         145
  C:034BH         LINE#         146
  -------         ENDPROC       _LCD_WDAT
  -------         PROC          LCD_INIT
  C:02E4H         LINE#         154
  C:02E4H         LINE#         155
  C:02E4H         LINE#         157
  C:02E6H         LINE#         158
  C:02E8H         LINE#         159
  C:02EAH         LINE#         160
  C:02F1H         LINE#         161
  C:02F6H         LINE#         162
  C:02F6H         LINE#         163
  C:02F9H         LINE#         164
  C:02F9H         LINE#         165
  C:02FCH         LINE#         166
  C:02FCH         LINE#         167
  C:02FFH         LINE#         169
  C:0301H         LINE#         170
  C:0304H         LINE#         172
  C:0309H         LINE#         173
  -------         ENDPROC       LCD_INIT
BL51 BANKED LINKER/LOCATER V6.05                                                      08/19/2015  12:09:32  PAGE 5


  -------         PROC          _LCD_POS
  D:0007H         SYMBOL        pos
  C:0003H         LINE#         182
  C:0003H         LINE#         183
  C:0003H         LINE#         184
  -------         ENDPROC       _LCD_POS
  -------         PROC          PLAY
  -------         DO            
  D:0007H         SYMBOL        i
  -------         ENDDO         
  C:0229H         LINE#         190
  C:0229H         LINE#         191
  C:0229H         LINE#         193
  C:022BH         LINE#         194
  C:022BH         LINE#         195
  C:0239H         LINE#         196
  C:023DH         LINE#         198
  C:0247H         LINE#         199
  C:0253H         LINE#         201
  C:0258H         LINE#         202
  C:025DH         LINE#         203
  C:0262H         LINE#         204
  C:0267H         LINE#         206
  C:026CH         LINE#         207
  C:0271H         LINE#         208
  C:0276H         LINE#         210
  C:027BH         LINE#         211
  C:0280H         LINE#         212
  C:0285H         LINE#         214
  C:028AH         LINE#         215
  -------         ENDPROC       PLAY
  -------         PROC          MAIN
  -------         DO            
  D:0004H         SYMBOL        m
  -------         ENDDO         
  C:000EH         LINE#         221
  C:000EH         LINE#         222
  C:000EH         LINE#         225
  C:0011H         LINE#         226
  C:0017H         LINE#         227
  C:001BH         LINE#         229
  C:001EH         LINE#         231
  C:0023H         LINE#         232
  C:0025H         LINE#         233
  C:002CH         LINE#         235
  C:0031H         LINE#         236
  C:0033H         LINE#         237
  C:0033H         LINE#         238
  C:003CH         LINE#         239
  C:0043H         LINE#         240
  C:0047H         LINE#         242
  C:004EH         LINE#         244
  C:0053H         LINE#         245
  C:0055H         LINE#         246
  C:0062H         LINE#         248
  C:0062H         LINE#         249
  C:0062H         LINE#         250
BL51 BANKED LINKER/LOCATER V6.05                                                      08/19/2015  12:09:32  PAGE 6


  C:0068H         LINE#         251
  C:0068H         LINE#         252
  C:006AH         LINE#         253
  C:006DH         LINE#         254
  C:0074H         LINE#         256
  C:0084H         LINE#         257
  C:0084H         LINE#         258
  C:0084H         LINE#         259
  C:0086H         LINE#         260
  C:008BH         LINE#         261
  C:008DH         LINE#         262
  C:009CH         LINE#         263
  C:009CH         LINE#         265
  C:009CH         LINE#         266
  C:009EH         LINE#         267
  C:00A3H         LINE#         268
  C:00A5H         LINE#         269
  C:00B4H         LINE#         270
  C:00B4H         LINE#         272
  C:00B4H         LINE#         273
  C:00B6H         LINE#         274
  C:00BBH         LINE#         275
  C:00BDH         LINE#         276
  C:00CCH         LINE#         277
  C:00CCH         LINE#         279
  C:00CCH         LINE#         280
  C:00CEH         LINE#         281
  C:00D3H         LINE#         282
  C:00D5H         LINE#         283
  C:00E4H         LINE#         284
  C:00E4H         LINE#         286
  C:00E4H         LINE#         287
  C:00E6H         LINE#         288
  C:00E6H         LINE#         289
  C:00E6H         LINE#         290
  C:00E6H         LINE#         291
  C:00E9H         LINE#         292
  C:00E9H         LINE#         293
  C:00EBH         LINE#         294
  C:00EEH         LINE#         295
  C:00EEH         LINE#         296
  C:00F7H         LINE#         297
  C:00FCH         LINE#         298
  C:00FEH         LINE#         299
  C:0105H         LINE#         300
  C:0108H         LINE#         301
  C:010FH         LINE#         302
  C:010FH         LINE#         304
  C:0112H         LINE#         305
  -------         ENDPROC       MAIN
  -------         PROC          TIME0
  C:028FH         LINE#         313
  C:0293H         LINE#         315
  C:0296H         LINE#         316
  C:0299H         LINE#         318
  C:029BH         LINE#         320
  C:02A0H         LINE#         321
BL51 BANKED LINKER/LOCATER V6.05                                                      08/19/2015  12:09:32  PAGE 7


  C:02A0H         LINE#         322
  C:02A3H         LINE#         323
  C:02A5H         LINE#         324
  C:02A5H         LINE#         325
  C:02AAH         LINE#         326
  C:02AAH         LINE#         327
  C:02ADH         LINE#         328
  C:02AFH         LINE#         329
  C:02AFH         LINE#         330
  C:02B4H         LINE#         331
  C:02B4H         LINE#         332
  C:02B7H         LINE#         333
  C:02B9H         LINE#         334
  C:02B9H         LINE#         335
  C:02BEH         LINE#         336
  C:02BEH         LINE#         337
  C:02C1H         LINE#         338
  C:02C3H         LINE#         339
  C:02C3H         LINE#         340
  C:02C8H         LINE#         341
  C:02C8H         LINE#         342
  C:02CBH         LINE#         343
  C:02CDH         LINE#         344
  C:02CDH         LINE#         345
  C:02D2H         LINE#         346
  C:02D2H         LINE#         347
  C:02D5H         LINE#         348
  C:02D7H         LINE#         349
  C:02D7H         LINE#         350
  C:02DCH         LINE#         351
  C:02DCH         LINE#         352
  C:02DFH         LINE#         353
  C:02DFH         LINE#         354
  -------         ENDPROC       TIME0
  -------         ENDMOD        1602_MIAOBIAO

Program Size: data=25.0 xdata=0 code=927
LINK/LOCATE RUN COMPLETE.  0 WARNING(S),  0 ERROR(S)
